:04000000B601C42958
:100008000800B616B61EB612B6190E28B615472041
:10001800031835280830A3005B20A20DA30B102875
:10002800B61E402065206120B61A35203A202208E5
:100038000310BF29B616B61EB61236192828FE397F
:10004800B70036150310BF29361A3028A600361611
:1000580047200318352826084E2003183528B61ED1
:10006800BF294020652036113612B6113A0884009F
:1000780038088417800446283A088400380980051F
:100088008417800508003A20652040206120370841
:10009800B6190138A2000830A300A20D03183A20AF
:1000A800031C402065206120A30B51283A206520BD
:1000B8003A08840038080005FF3E3B0884003909E7
:1000C80043283B08840039083D282C08A0002D0847
:1000D800A1000130A20064009520031C8228A20B15
:1000E8006F28FF30A007031CA107031CBF29FA30A3
:1000F800A2006F286400952003187E28E720A80135
:100108000830A300E82095200318A80AAB1EA80110
:10011800A20CA30B8628AB1AA213E820031422080A
:1001280008003A08840038088417800484130005FE
:100138002B1B3806FF3E0800A400290803140319E6
:10014800BF29BA21031C0800A0002518831724081A
:100158008400200880008313A40AA903A1280408A6
:10016800A6003A088400F030B7050830A70003104D
:100178000318B70ACD20A60CA70BBC280000AB1AA1
:10018800370CCD20C2210314CD202F08A3002E0840
:1001980039298413AB1FDC28000838042B1F3806C4
:1001A8008000841700083804031C38068000E828FB
:1001B80000083804031C38062B1B380680008417F7
:1001C80038098005E82837172B081F39003EA10099
:1001D8002A080E3E0318A10A371F46293713A00024
:1001E800023060214629B71329080319B7170430CC
:1001F800A800250E042125080421240E0421240822
:100208000F39F63E0318073E0A3E2729B713290877
:100218000319B7170530A8002730A3001030202194
:100228000330A300E8302021A30164302021A3017A
:100238000A30202124082729A2002508A100240823
:10024800A00088212008A000A8030319B7132908D3
:10025800031931292802031808002008031DB713C1
:10026800B71B0800303EBA29A301A200FF30A2073D
:10027800031CA307031CBF290330A100E730462154
:100288003A29A101FC3EA000A109031C5129FF3015
:100298000000A00703184C29A0076400A10F4B29F0
:1002A80008000310A00DA10DFF3E031855292008D2
:1002B800BF290310A10CA00CFF3E03185D292008DC
:1002C800BF29A301A20001307129A301A2000630B1
:1002D8007129A101A301A2000530A8002308210269
:1002E800031D78292208200204300318013003195D
:1002F80002302805031DFF30BF290038031DFF30D9
:100308000405031DFF30BF291030A600A501A40174
:10031800210DA40DA50D2208A4022308031C230FF8
:10032800A50203189E292208A40723080318230FEF
:10033800A5070310A00DA10DA60B8C292008BF2925
:100348001030A800A101A001A70CA60C031CB2291B
:100358002208A00723080318230FA107A10CA00C4B
:10036800A50CA40CA80BA8292408BF2984003108CF
:100378008A00300882008313031383126400080084
:10038800831607309F009901831298018316023063
:1003980098000610861006118801871007100711AB
:1003A800871205128512C001B4010130BF00D701C0
:1003B800C430D600831288018614061587140715E1
:1003C80087120714851206100130A300F4308A0141
:1003D80039218316A6011030A700AA01AB016400D9
:1003E8008A110A128312871A082A83160830AD0068
:1003F8000730AC002030A400A5012030A800A901D6
:1004080083128A110A12142A83160630AD000530A9
:10041800AC002830A400A5012830A800A901831247
:10042800071001308A01382107148A110A12AF2EE9
:100438008A110A12432283164D0883128800071175
:10044800061587108610861487148A110A1243220B
:1004580083164E0883128800071106158710861028
:10046800861487148A110A12432283164C088312B1
:1004780088000615871086108614871408008714CC
:100488008316FF308800831207158614871006111B
:10049800003008180130A00001308A016D21B20037
:1004A800003088180130A00001308A016D21B400A5
:1004B8003208840034088A0181218A110A12031D36
:1004C800432A0615871483168801831208008A01B7
:1004D80043228316FF308800831207118614061101
:1004E800871002308A01452108088316B20083125A
:1004F8008714061583168801831208008A110A12C8
:10050800242383165608CC0083128A0136228A01D6
:100518006B22080083160130D70083128316200847
:100528008312A600831621088312A7002030A20098
:10053800A3018A01A421B2002508B3008316260866
:100548008312B207831627080318013E8312B307E4
:100558007D08A0007E08A10083162D088312A20042
:10056800A3018A018821B4002108B50032083407A4
:10057800F50033080318013E3507F6007508FB003F
:100588007608FC007D088316BD002008BE00831293
:1005980076088316CE00831275088316CD002430A2
:1005A800CC0083128A011C22640083165708003C81
:1005B8008A110A128312031D012B7D08A0007E08F0
:1005C800A10083162D088312A200A3018A018821A5
:1005D8002408B2002508B300320883162C028312BF
:1005E800B20033090318013EB300F8303204831611
:1005F800CC0083128A110A121E2B7D08A0007E08E7
:10060800A10083162D088312A200A3018A01882164
:100618002408B2002508B300320883162C0283127E
:10062800B20033090318013EB300F03032048316D8
:10063800CC0083128A0136228316D7018312080060
:10064800831620088312A600831621088312A700A8
:100658002030A200A3018A01A421B2002508B3001A
:10066800831626088312B207831627080318013E4B
:100678008312B3077D08A0007E08A10083162D0809
:100688008312A200A3018A018821B4002108B500C1
:1006980032083407F50033080318013E3507F60021
:1006A8007508FB007608FC0076088316CE008312D6
:1006B80075088316CD002430CC0083128A011C22D1
:1006C800080083164A0847078312FD00FE01FE0D45
:1006D80083164B084807A000A101A10D83128A01C7
:1006E800922283164A0847028312FD00FE01031C6A
:1006F800FE0383164B084807A000A101A10D831231
:100708008A019222831647084A078312FD00FE01D8
:10071800FE0D83164B084802A000A101031CA1038B
:1007280083128A01922283164A0847028312FD0027
:10073800FE01031CFE0383164B084802A000A1011A
:10074800031CA10383128A01922283164B084707D0
:100758008312FD00FE01FE0D83164A084807A0001B
:10076800A101A10D83128A01922283164B08470228
:100778008312FD00FE01031CFE03831648084A0786
:10078800A000A101A10D83128A01922283164708B5
:100798004B078312FD00FE01FE0D83164A0848022E
:1007A800A000A101031CA10383128A0192228316CF
:1007B8004B0847028312FD00FE01031CFE0383164B
:1007C8004A084802A000A101031CA10383128A0160
:1007D8009222080083162708CE002608CD00423052
:1007E800CC0083128A011C2283162508CE00240817
:1007F800CD004330CC0083128A011C2283162B08BB
:10080800CE002A08CD004030CC0083128A011C2279
:1008180083162908CE002808CD004130CC00831269
:100828008A011C2283168030CC0083128A0136226A
:100838008316CE01CD012430CC0083128A011C22FC
:1008480083169830CC0083128A0136228316013031
:10085800B40083126400F130831634028A110A123C
:1008680083120318592C83160130B80083126400D0
:100878004130831638028A110A1283120318522C47
:100888008316CE01C030CC0083128A012922831638
:10089800B80A8A110A128312031D3B2C8316B40A64
:1008A8008A110A128312031D2E2C08008316CA010E
:1008B8004908CB000310490D8312B200B301B30DF0
:1008C8003208023C8316A20083123308031C013E3F
:1008D800003C8316A3008312640083164A084B0267
:1008E8008A110A128312031CCB2C8A016523640027
:1008F8008A110A1283168310A31F83148312831884
:10090800A32C0430A600A70183164A088312A2006C
:10091800A3018A01A421B2002508B3000630B2075A
:100928000318B30A32088316A20783123308031880
:10093800013E8316A30783128A110A12C62C831656
:100948004B084A028312B200B301031CB3030430FC
:10095800A600A7013208A2003308A3008A01A42137
:10096800B2002508B3000A30B2070318B30A3208E8
:100978008316A207831233080318013E8316A307C0
:10098800CB0383128316CA0A83128A01702C0800CB
:100998008A110A12C825831641084202BA0044087F
:1009A8004502BB0064003B083A028A110A1283120E
:1009B800031C4F2D83163B088312A000A1010230AF
:1009C8008A015821B2002108B30083163A0883121D
:1009D80032028316A20083123308031CFF3E8316DB
:1009E800A3004408A000A1013B088312A000A101B4
:1009F80002308A015821F7002108F80083163A08C6
:100A08003B028312B200B301031CB3030310320D7F
:100A1800F900330DFA00831641088312FD00FE0128
:100A28007D08A0007E08A1008316420883128A016F
:100A380065218A110A12031D4E2D64008A110A12BB
:100A480083168310A31F831483128318382D770805
:100A58008316A207831278080318013E8316A3079A
:100A680083128A110A12452D79088316A207831268
:100A78007A080318013E8316A307A00A0319A10ADE
:100A880083128A019222FD0A0319FE0A8A110A12A8
:100A9800031D142D080083163A088312A000A10133
:100AA80002308A015821B2002108B30083163B089E
:100AB800831232028316A20083123308031CFF3EFE
:100AC8008316A30041088312FD00FE0183163A082D
:100AD8008312A000A10102308A015821F7002108E1
:100AE800F80083163B083A028312B200B301031CD4
:100AF800B3030310320DF900330DFA0083164408CE
:100B0800A000A1018312831620088312A000831677
:100B180021088312A1008316450883128A016521E2
:100B28008A110A12031DC72D64008A110A1283163E
:100B38008310A31F831483128318AF2D770883169D
:100B4800A207831278080318013E8316A3078312AD
:100B58008A110A12BC2D79088316A20783127A0813
:100B68000318013E8316A3078312FD0A0319FE0A20
:100B78008A0192228316A00A0319A10A8A110A126D
:100B88008312031D872D0800640083164108420262
:100B98008A110A1283120318D72D831641084202BC
:100BA800C107C202831264008316440845028A11F1
:100BB8000A1283120318E62D831644084502C40757
:100BC800C50283120800831620088312A00083162A
:100BD80021088312A1000830A200A3018A018821FC
:100BE800B2002108B3003208A6003308A70020305D
:100BF800A200A3018A01A421B2002508B30083162C
:100C08002A088312B20783162B080318013E8312A1
:100C1800B3077D08A0007E08A10083162D08831263
:100C2800A200A3018A018821B4002108B500320876
:100C38003407F50033080318013E3507F600760837
:100C48008316CE00831275088316CD002430CC009D
:100C580083128A011C22080020308316B1028312F5
:100C68008A110A1257268A01E72583163108CE0011
:100C78005608CC0083128A0129228A110A125E269C
:100C880008008A01242383163008CE005608CC00B9
:100C980083128A012922080083169830CC00831217
:100CA8008A013622080083169430CC0083128A0108
:100CB8003622080083169C30CC0083128A01362223
:100CC8000800831637083C3E840000088312B200EF
:100CD800FF30A200A20A22080F3C8A110A12031C44
:100CE800982E8A110A12842632028A110A12031DCA
:100CF8006E2E22088316CF0083128A110A12982EAC
:100D080006308A00220882073034313432343334D2
:100D18003434353436343734383439346134623421
:100D28006334643465346634080083162708CE00BB
:100D38002608CD004230CC0083128A011C2208000C
:100D480083162B08CE002A08CD004030CC00831231
:100D58008A011C2208008A01EE238A015026831684
:100D68007730C7001F30C8001430C9000A30C900E6
:100D7800831264001A30831649028A110A128312F8
:100D88000318D02E8A015A2405308316C9078A1100
:100D98000A128312031CBD2EFD01FE0183161830B2
:100DA800A000A101C030D600B401831264001E3037
:100DB800831634028A110A1283120318282F831605
:100DC80034081D3C8A110A128312031C1F2F8A1132
:100DD8000A12F4268316B10083128A110A121F2FF1
:0C0DE80007308A00831634088312002FA5
:100E0000820754344F3453344834493442344134E3
:100E10002034543436343934363433342034443482
:100E200065346D346F34203466346F34723420345A
:100E300047344C34693450344934433432348A01B1
:100E400030268316B40A8A110A128312031DDA2E81
:100E50008316C101EF30C200C401C50183128A01AB
:100E6000CC248A110A12D92FF301F401FD01FE01ED
:100E70007D08A0007E08A1000730A3007F308A0112
:100E800066218A110A12031D6C2F8316AB30B00045
:100E900007308312BA001030B8000730BB000830AA
:100EA000B900A0308A01202074088A01202073082C
:100EB0008A0120208316300883128A011E200A30FE
:100EC0008A013821F30A0319F40AFD0A0319FE0AFC
:100ED0008A110A12031D382F8A110A12D62FF30124
:100EE000F4018316A001A101831283162008831246
:100EF000A000831621088312A100A3013F308A01BC
:100F000066218A110A12031DD62FFD01FE017D08FC
:100F1000A0007E08A100A301EF308A0166218A119A
:100F20000A12031DCD2F0730BA001030B800073069
:100F3000BB000830B900A0308A01202074088A0163
:100F4000202073088A0120208A0105208316B00022
:100F500007308312BA004030B8002030AA00AB013D
:100F6000AE01AF01A901831630088312A400A501C8
:100F7000B330B000B1018A01F7208A014526F30A97
:100F80000319F40A0830FD078A110A12031C872F7F
:100F9000FE0A8A110A12031D872F8316A00A03195D
:100FA000A10A8A110A128312031D752F64008A0197
:100FB000D62F8316B801B701B90183122030FF0084
:100FC00083160A30B3008312F501F601FD01FE011C
:100FD0008316A001A10183128A0150268316C43012
:100FE000D6007830B500B6018312F301F401073062
:100FF000BA008030B8002030AA00AB018A017E2000
:101000002A3C8A110A12031DFE2F0930A9007E30E6
:10101000B000B101A5016B308A01A0208316B70191
:10102000831264000930831637028A150A1283126C
:1010300003185928831637086B3E84000008831272
:10104000B200FF30A200A20A22080F3C8A150A1241
:10105000031C4D288A150A12392032028A150A12F9
:10106000031D232822088316CF0083128A150A1233
:101070004D2808308A002208820730343134323457
:1010800033343434353436343734383439346134E5
:1010900062346334643465346634831637086B3ED7
:1010A00084004F088000B70A8A150A128312031DB4
:1010B00011287208A000A10104308A015821B20051
:1010C0002108B300730832048316B30083126C083E
:1010D000A000A10104308A015821B2002108B30008
:1010E0006D083204FF006E08A000A10104308A01DF
:1010F0005821B2002108B3006F083204F6007008CE
:10110000A000A10104308A015821B2002108B300D7
:1011100071083204F5000730BA004030B8002030C2
:10112000AA00AB01AE01AF0144308A01B42069309E
:101130008A01B42073308A01B42070308A01B4204F
:101140006C308A01B42061308A01B42079308A0180
:10115000B42065308A01B42064308A01B420A9012A
:101160007F08A400A501B330B000B1018A01F720C7
:10117000A901831633088312A400A501B330B0007F
:10118000B1018A01F7200A308A01B4200D308A01AA
:10119000B4207508F3007608F4006B088316B800D5
:1011A00064003808003C8A150A1283120319752A54
:1011B000640083163808013C8A150A128312031949
:1011C0000529640083163808043C8A150A12831224
:1011D0000319F528640083163808053C8A150A129D
:1011E00083120319DF298A01F72F8316E830B5002F
:1011F000B6018312FD01FE018316A001A101831235
:10120000F301F4018A150A12822A0730BA008030ED
:10121000B8002030AA00AB018830AC001330AD001C
:101220008A0169208A150A12031C402B5D3C8A152D
:101230000A12031D10297F08A9006930B000B1010E
:10124000A5013C308A01A0208A150A12031C402BFC
:101250008316B7018312FF307F07B400FF300318F5
:10126000013EB500831637088312A000A10135089E
:10127000A30034088A0166218A150A12031D7F29FA
:10128000831637083C3E840000088312B200FF300A
:10129000A200A20A22080F3C8A150A12031C732915
:1012A0008A150A125F2132028A150A12031D492982
:1012B00022088316CF0083128A150A127329093077
:1012C0008A002208820730343134323433343434E3
:1012D0003534363437343834393461346234633435
:1012E000643465346634831637083C3E84004F0806
:1012F0008000B70A8A150A128312031D2B29831650
:10130000B7018312FF307F07B400FF300318013E9E
:10131000B500831637088312A000A1013508A30089
:1013200034088A0166218A150A12031DDC298316F6
:1013300037083C3E840000088312B2003208A00047
:10134000A10104308A015821B2002108B300013004
:10135000831637078312B400B501B50D34083C3E3F
:1013600084000008B400340832048316B00007304B
:101370008312BA001030B8000730BB000830B90043
:10138000A0308A01202074088A01202073088A0175
:1013900020208316300883128A011E200A308A0119
:1013A0003821F30A0319F40A02308316B7078A15A5
:1013B0000A128312031C82298A150A1205297F0842
:1013C000A600A7010830A200A3018A01A421B2004F
:1013D0002508B30032038316B5003303B600831229
:1013E000FD01FE018316A001A101C430D600A001B9
:1013F000A1018312831620088312A00083162108FE
:101400008312A1008316360883128A0165218A158A
:101410000A12031D492AFD01FE017D08A0007E0875
:10142000A1008316350883128A0165218A150A12E4
:10143000031D402A0730BA001030B8000730BB0047
:101440000830B900A0308A01202074088A012020C9
:1014500073088A0120208A0105208316B0008312B8
:101460008A014526F30A0319F40A0830FD078A1594
:101470000A12031C0D2AFE0A8A150A12031D0D2AE0
:101480008316A00A0319A10A8A150A128312031DE2
:10149000FA290730BA004030B8002030AA00AB016A
:1014A000AE01AF0144308A01B42069308A01B42012
:1014B00073308A01B42070308A01B4206C308A0104
:1014C000B42061308A01B42079308A01B4206530BB
:1014D0008A01B42064308A01B4200A308A01B42021
:1014E0000D308A01B4208A01F72F8A0199268316CC
:1014F000E830B500B6018312FD01FE018316A0019C
:10150000A10183120730BA008030B8002030AA0051
:10151000AB01D030AC000730AD008A0169208A11E0
:101520000A12031CF72F5D3C8A150A12031D8D2A2F
:101530007F08A9006930B000B101A5013C308A01E3
:10154000A0208A110A12031CF72F8316B7018312F9
:10155000FF307F07B400FF300318013EB50083164B
:1015600037088312A000A1013508A30034088A01BE
:1015700066218A150A12031DCB2A8A016526831665
:1015800037083C3E84004F088000B70A8A150A12CB
:101590008312031DA82A8316B7018312FF307F0729
:1015A000B400FF300318013EB500831637088312DC
:1015B000A000A1013508A30034088A0166218A151C
:1015C0000A12031D3D2B831637083C3E8400000899
:1015D0008312B2003208A000A10104308A01582110
:1015E000B2002108B3000130831637078312B4001C
:1015F000B501B50D34083C3E84000008B400340841
:1016000032048316B00083127D08A0007E08A1007A
:101610008316350883128A0169218A150A12031D6F
:101620001B2B831636088312FD00FE018316A00AC9
:101630000319A10A8312831620088312A0008316BF
:1016400021088312A100A3013F308A016A218A1573
:101650000A12031D2F2B8316A001A10183128A01F8
:1016600045260830FD070318FE0A02308316B70727
:101670008A150A128312031CCE2A8A150A12822A9C
:101680000730BA004030B8002030AA00AB01AE01EC
:10169000AF016C308A01B42061308A01B42073300C
:1016A0008A01B42074308A01B42020308A01B42029
:1016B00062308A01B42079308A01B42074308A0102
:1016C000B42065308A01B42020308A01B420613012
:1016D0008A01B42074308A01B4203A308A01B420DF
:1016E000A9017308A4007408A500B330B000B101CB
:1016F0008A010A210A308A01B4200D308A01B420FF
:0C1700008A01F72F63008A150A12822B61
:02400E00753DFE
:00000001FF
